:020000000628D0
:080008000B11090005308C000A
:1000100009308D000A308E0006308F0083160030C4
:1000200086008312003098000130003C03192D280F
:1000300018080C3E84000008860014309300372016
:100040001808980A1808043C0130031D0001003C00
:1000500003192C280030980014281008910014303F
:10006000920000000000920B3128910B2F281308FA
:1000700095006E30940000000000000000000000B9
:100080000000940B3B28950B392808001608003C0B
:10009000013003190001003C03196028003097006B
:1000A0000A301702013003180001003C03195D28D3
:1000B000643093003720970A502816089603462884
:0200C000080036
:00000001FF
